:0400000000000428D0
:080008008A110A120728E130F9
:10001000831603138600831286016E2032305C2023
:100020000230831203138600013083120313060586
:1000300083120313A2002208031D1428A201043016
:1000400083120313220203182D2802308312031394
:10005000860632305C20A20A1F28C03083120313A8
:10006000060583120313A0002008403A0319412813
:100070002008803A031948282008C03A03194F285D
:1000800056281E3083120313860032305C202D2840
:10009000143083120313860032305C202D28163072
:1000A00083120313860032305C202D281C3083120B
:1000B000031386002D28080083120313A1002108D2
:1000C00003196D283D308312031381000B110B1DA2
:1000D000672883120313A1035F2808008730831663
:0600E0000313810008007B
:02400E00FF3F72
:00000001FF
